:020000040000FA
:100000008501073099005828A900030EAA000108AD
:10001000AD000408AB008B1C342881018B1005193E
:1000200017280B118B16831601178312512883167C
:10003000011383128B1E51282C148B1264302D0255
:10004000031C2528E030AF003A2808302D02031C9D
:1000500051283008840027302D02800DAF0F312841
:100060002C10AE0F512845288B1E51280B1D5128EE
:100070008B122C10F8302E02031951282C1730083F
:1000800084000310800DAE0F4128F830AE00B00A96
:100090006030300247300319B000300826020319DF
:1000A000AC162B0884002A0E8300A90E290E090025
:1000B0004730B000A60084008001F830AE003A302E
:1000C000B800B9008316443081000E30850064000A
:1000D000FF2390008312AC01B501B301C601BE300D
:1000E000A200FE30A3001322F52190308B008E2257
:1000F00043309122523091221010CF308F002B309C
:100100008E000C10313090001722B50A03198E2290
:10011000B70F8E28CE30B700FB30AC05B60FB32832
:10012000F630B600C608031DC603AC1DB128A503F2
:100130000F302505FB3EFA300319A507A63025022E
:100140000318B328FF30A500A4030F302405FB3E9D
:10015000FA300319A407663024020318B328FF30CD
:10016000A4000C187C28AC1EB928AC1203309122D4
:100170008C222C1FBF282C13003091228C22C60801
:100180000319DC2039088400C608031DB128380291
:100190000319B128AE220319C2288318D5284B228F
:1001A0002C18B1284F22800AB1284B222C18B128D4
:1001B0006722800A800AB12826088400E2210319F8
:1001C0000800533027020319E9282708A222262114
:1001D000DE28E221031908002C3027020319F32836
:1001E0005330A222E128E221031908002708A800C1
:1001F000E2210319080027082807013E031D0F29E3
:1002000028080339031D0F292621FC30B3000330D1
:100210008A000310A80C280CA80DBF3E82002608F7
:100220008400E221031908002708A222E221031911
:1002300008002708A222E221031908002708A222A9
:10024000E221031908002708A2228C220408A60034
:100250000800753091222808A222753091228C2A3C
:10026000B30108000B3091228C22AC1D3B298A225D
:10027000973091220800FF218A22923091227A3011
:1002800091228A22923091228A229730912208006C
:10029000AC19FF211322133091228C2AAC19F121C1
:1002A000BE30A2008A2292309122063091220E3076
:1002B00091228C22773091228A2297309122080055
:1002C0001322A20ABF302202BE300318A2008A22E3
:1002D0008D3091221C309122233091228C2A1322BE
:1002E000A203B9302202B930031CA2008A2288304E
:1002F0009122203091228C2A0230AC0629309122A2
:100300008C2A0430AC06CE30B7008A22923091227B
:10031000303091228C228A22973091220800AC1929
:100320000D221322A3030F302305FB3EFA300319DD
:10033000A30766302302FE30031CA3008A22883004
:1003400091228A2297309122353091228C2AAC1941
:100350000D221322A30A0F30230506300319A30729
:10036000FF30230266300318A3008A228D309122C9
:100370008A22973091223A3091228C2ABE30A200F4
:100380009022573091228C2ABD30A2009022593001
:1003900091228C2ABC30A20090225B3091228C2AC0
:1003A000BB30A20090225D3091228C2ABA30A2008C
:1003B00090225F3091228C2AB930A20090226130C5
:1003C00091228C2A04083002031908000008A700B3
:1003D000840A60300402031D0800473084000311C2
:1003E0000800AC11B430B1000800AC11BB30B10052
:1003F000EC30B2000800AC15F530B1000800AC15C7
:10040000BF30B1002E30B400E830B2000800AC15A7
:10041000D730B100F630B2000800AC15EB30B100B7
:10042000F430B2000800FF30A500A400080002303C
:100430008A00310882002208362223083622240846
:10044000362225083622FB30AC1C0F382C192F39E8
:10045000362A6630362266303622A6303622B7304B
:10046000362AB3080319362ADF39B30A4B22A10A08
:10047000050820388500EF39A00D031810388500D5
:10048000DF398500AD23AD23A10F392A5130013E5C
:10049000031D472A0800A000F730A10008008B13B5
:1004A0000508013885009F23AB23A10A0319602AA0
:1004B000A00C031C512AFE398500AB23AB23552A1F
:1004C000612AFE3985008B179F239F230800851022
:1004D0008B13831685108312AB23AB23A10A031958
:1004E0007A2AA00C031C692A831685148312A02380
:1004F000AB236E2A7B2A8316851483128B17AB23BA
:100500009F230800B90A463039023A300319B9006E
:10051000031508007D30912A5230912A4830912AE3
:100520002430A0000408A1003808840020088000BE
:10053000B80A463038023A300319B800210884005E
:1005400003150800A800280E0F39A1002107553E09
:100550009122A80D28081E39553E912A03308A00A1
:100560000008031183108200743031221B228F3067
:1005700036227C30312AB20FB42AFF21B42A34301B
:100580003122321CCB2A1B22EF3036223C30312262
:10059000B20F0800072A34083622293034022E30E0
:1005A000031D3403B4002922FF303622C62A34301A
:1005B0003122321CE32A1B22AE3036223C3031225B
:1005C000B20F0800FB2922080F39203836222922D1
:1005D000FF303622DE2A343031221B22AE30362262
:1005E0003C303122B20F0800FB29343031221B226B
:0805F000CF3036223C30312AE5
:1006000064346534822A6F346634822A4D3444342B
:1006100049345334822A4D3445344E3441344234C3
:100620004C344534822A4D3449344E345134553497
:10063000493452345934822A503452345634822A3E
:100640004E34583454345F344C3449345334543475
:10065000822A523441344E3444344F344D34822A49
:1006600050344C3441345934822A4E344534583451
:100670005434822A503452344534563449344F3439
:1006800055345334822A523449344E344734822A02
:100690005634573443344434503449344334323478
:1006A0002E3438340D340A34822A3034822A3134DC
:1006B000822A3234822A3334822A3434822A3534EC
:1006C000822A3634822A3734822A3834822A3934CC
:1006D000822A4134822A4234822A4334822A443490
:1006E000822A4534822A4634822A2D34822A0330D3
:1006F000C600822A0130C600822A8314FF34831484
:100700005534831403348314023483140034822A4E
:10071000831408348314F334822A8314103483142A
:10072000EB34822A831401348314FA34822A00348D
:10073000831400348314FB34822ABB049F2BA02B28
:10074000A12BA22BA32BA42BA52BA62BA72BA82B2D
:0E07500008000000A02B0000A12B0000A42B2D
:02077E00292927
:1007800029292929BE294E293029602929292929E1
:1007900029292929D62929292929482929292929FD
:1007A00029292929CA2929292929602929297C298E
:1007B00029298F29292929292929A72929292929C5
:1007C00029292929C42929292929292929298129A6
:1007D0002929A729DC292929292929292929292958
:1007E00029292929D029292929296F2929297C2939
:0E07F000322929292929292929298F2929294E
:02400E00C43FAD
:10420000560057004300440050004900430020007E
:104210004600690072006D00770061007200650061
:104220002000760032002E00380070007200650019
:1042300033000A0043006F007000790072006900CB
:104240006700680074002000280063002900200037
:1042500032003000300032002D00320030003000DB
:1042600034002C002000450064002000530063004F
:1042700068006C0075006E0064006500720020002C
:104280003C006500640040006B0039007300700062
:10429000750064002E0063006F006D003E000A0090
:1042A0004C006900630065006E00730065006400E7
:1042B000200075006E006400650072002000470059
:1042C0004E0055002000470065006E00650072003A
:1042D00061006C0020005000750062006C006900F5
:1042E000630020004C006900630065006E007300ED
:0C42F00065002000760032002E000A005D
:00000001FF
